:020000020000FC
:100000000C9413011895189518951895189518952E
:100010001895189518951895189518951895189578
:100020001895189518951895189518951895189568
:100030001895189518951895189518951895189558
:100040001895189518951895189518951895189548
:100050001895189518951895189518951895189538
:10006000189518951895189500E005B90FEF04B983
:1000700000E008B90FEF07B900E00BB90FEF0AB9BC
:100080009FD080D001D0FFCF9A938A9380E090E0F8
:1000900031C011E001E035D011E001E032D011E0D3
:1000A00002E02FD011E002E02CD011E004E029D0D2
:1000B00011E004E026D011E008E023D011E008E0D0
:1000C00020D011E000E11DD011E000E11AD011E0D4
:1000D00000E217D011E000E214D011E000E411D0EA
:1000E00011E000E40ED011E000E80BD011E000E8D0
:1000F00008D00196833300E0900758F289919991D6
:1001000008959A938A93902F812F01E010E066D092
:10011000813011F45E9A01C05E9801E010E05ED07B
:100120005D9801E010E05AD09EBD0DB5102F17FF6D
:10013000FCCF01E010E052D05D9A01E010E04ED01B
:100140008991999108955E9A01E010E047D05D9AF7
:1001500001E010E043D05C9801E010E04AD05C9AE6
:1001600001E010E046D008955C98549A5F98579A41
:10017000559A569A04E610E03CD05F9A04E610E0E7
:1001800038D00895F1DFDFDF08EE13E027D010E06C
:1001900001E2B7DF10E009E0B4DF10E000EEB1DF0C
:1001A00010E006E1AEDF10E006E0ABDF10E000E2B9
:1001B000A8DF10E00CE0A5DF08EE13E00FD00895F3
:1001C00000E005B9239A259A229A00E00DBD03E5C7
:1001D0000CBD02E310E00DD00DB508959C01C801DF
:1001E00003C0A89500000197082F092BD1F7C9017A
:1001F00008959A938A93C80104C008EE13E0EEDFD5
:100200000197082F092BC9F78991999108950895AD
:100210002297C801888399839E0101E00E9407010B
:10022000F9CF0C9408010FE30DBF01E00EBFC0E24F
:10023000D1E00E9423010E9434000E9421010C940D
:0A02400011010C94110101E0089572
:0400000300000000F9
:00000001FF
